:020000040000FA
:1000000083168E100E141528A5000308A7000408F7
:10001000A6000A08A8003A2028088A0026088400BA
:1000200027088300A50E250E0900FF239000183035
:100030009F0083128501073099000C309F008316C2
:1000400038308500573081008312203084008001D1
:10005000840A29300402031D27280030A3000C3035
:10006000A2001430A100F0308100A0308B0000000D
:10007000000037280B1D0800F03081000B11A2088A
:1000800003194428A2036828A10B68280C30A20099
:100090002008A100A10CA10C3F30A105A10A00304D
:1000A0002306031D55280130662801302306031D51
:1000B0005B280330662803302306031D61280730C0
:1000C000662807302306031D68280030A30085003A
:1000D0000D309F0073209F149F186C281E08A000ED
:1000E0000C309F0008000530A400A40B7528080000
:02400E00843FED
:00000001FF
